:103C00000C942A1E0C94481E0C94481E0C94481EBA
:103C10000C94481E0C94481E0C94481E0C94481E8C
:103C20000C94481E0C94481E0C94481E0C94481E7C
:103C30000C94481E0C94481E0C94481E0C94481E6C
:103C40000C94481E0C94481E0C94481E0C94481E5C
:103C50000C94481E11241FBE20E0A89521BD20E031
:103C600025BF20E026BFE6E7FFE3A0E6B0E020E0C6
:103C700002C005900D92A036B207D9F7A0E6B0E0D9
:103C800020E001C01D92A036B207E1F70C944B1E54
:103C90000C944A1E1895CFE5D4E0DEBFCDBF8BE073
:103CA00089B988E18AB9949A80B384FD30C10E94B1
:103CB000921F982F913609F426C1913409F412C14C
:103CC000933609F40BC1933409F4F9C09E3609F414
:103CD0001AC19D3409F4C6C0953609F4B6C09C36A5
:103CE00009F4AEC09D3609F4A6C0903509F407C1A9
:103CF0009C3409F404C1903709F499C0923509F451
:103D000088C0943409F478C0943609F469C09634B4
:103D100009F45EC0923709F457C09E3409F450C0CC
:103D2000943709F446C0892F8857823018F40E94CE
:103D3000921FE5C09435D9F3933529F19635E1F01A
:103D4000963799F0933739F09B3109F4B0CF8FE370
:103D50000E948C1FACCF81E00E948C1F84E90E94DE
:103D60008C1F8EE10E948C1FA2CF81E30E948C1FCA
:103D700080E30E948C1F9BCF82E30E948C1F83E311
:103D80000E948C1F94CF81E40E948C1F86E50E94C4
:103D90008C1F82E50E948C1F82E40E948C1F8FE49E
:103DA0000E948C1F8FE40E948C1F84E50E948C1F50
:103DB0007ECF81E60E948C1F80E00E948C1F77CF0F
:103DC00069E083E090E007C069E081E090E003C033
:103DD00069E080E090E00E94A71F0E948C1F67CFDF
:103DE000CEBB8D2F99278FBB21968CB381608CBB66
:103DF0008DB30E948C1F5BCFCEBB8D2F99278FBBBD
:103E000021960E94921F8DBBE29A8CB381FDFDCF5B
:103E100076C060E0CE010E94A71F8C01812F9927F8
:103E20000E948C1F802F0E948C1F229640CF83E51A
:103E30000E948C1F3CCF65E0CE010E94941F5FC0A2
:103E40000E94921F0E94B21F5AC0C0E0D0E063E0FF
:103E5000CE010E94941FC058DF4F8CE3C030D807BA
:103E6000B0F34DC00E94921FF82E6E01EE24EF14A5
:103E7000A0F40E94921FB82E0B2D11270E94921FB2
:103E80009927982F8827082B192BBE01C8010E945B
:103E90009C1F2296E394EF1460F38F2D0E948C1FD9
:103EA0008D2D99270E948C1F8C2D0E948C1F8D2F89
:103EB00099270E948C1F8C2F0E948C1F20C00B2DD5
:103EC00011270E94921F9927982F8827082B192BBA
:103ED000BE01C8010E949C1F229611C00E94921F21
:103EE000B82E0DC00E94921FC82FDD27DC2FCC27D3
:103EF0000E94921F9927C82BD92BCC0FDD1F8DE074
:103F00000E948C1FD4CE89E50E948C1FD0CE0E94C7
:103F1000000080E090E0FFCF8CB98BB186FFFDCF31
:103F20005E9A0895FFCF089525D0F92FE82F67BF37
:103F3000E895FFFF00001EC01DD0F72FE62F192EB9
:103F4000082E21E027BFE895FFFF000013D012D014
:103F5000F92FE82F60FD67BFC895802DE395C895C0
:103F6000902D089507D0082E19E017BFE895FFFFA0
:063F7000000000D00895DE
:0400000300003C00BD
:00000001FF
